S12301000000000000000000000000000000000000000000000000000000000000000000DB
S1210120000000000000000000000000000000000000000000000000000000000000BD
S12350007E508A7E50D27E50E17E50F07E50FF7E510C7E51707E51D77E51F47E51FA7E523E
S1235020007E52017E520C7E52257E522B7E52317E52407E524B7E52777E52FB7E530D7E35
S123504053587E53597E535A7E535B70726F6772616D2061392E61736D20332D32302D39B7
S1235060352020686331312064617461206C6F6720746F207063202035206279746573209C
S1235080393630302062617564048E00FF8680B710398630B7102BBD5240CE504BBD52FB80
S12350A0BD5201BD5201BD51D7010101BD50FF8603BD5261B61031BD5261B61032BD526110
S12350C0B61033BD5261B61034BD5261BD523120DB39CE003218CE164E180926FC0926F5D4
S12350E039CE00FA18CE164E180926FC0926F539CE01F418CE164E180926FC0926F539CE46
S123510010308614A7001F0080FC4F3918CE000ACC0000FD025ACC0000FD025CCC0000FDE2
S1235120025ECC0000FD0260BD50FFF610314FFD0258FC025AF30258FD025AF610324FFD75
S12351400258FC025CF30258FD025CF610334FFD0258FC025EF30258FD025EF610344FFD84
S12351600258FC0260F30258FD0260180926B939C640F71023FC1018F30113FD1018FE010F
S12351802D09FF012D27013BFE012FFF012DC680F71039CE10308614A7001F0080FC4FFE2D
S12351A00129B61031A700FC0129C30001FD0129FE0129B61032A700FC0129C30001FD0163
S12351C029FC0129B301271A8300002E022006FC0125FD01293B39CE00D918CE5200867E0E
S12351E0A7001AEF01CE00DC18CE5170867EA7001AEF0139C680F7103939C600F7100739EF
S12352003B860DBD5261860ABD526139CE1031BDFFBECE1032BDFFBECE1033BDFFBECE1097
S123522034BDFFBE398630B7102B398631B7102B39CE000118CE041A180926FC0926F5394D
S12352408600B7102C862CB7102D39A6008D04A600200444444444840F8B3081392F028B1D
S123526007F6102EC4C0C1C026F7F61000C404270220EEB7102F39CE528C18CE00C4C63C41
S1235280A60018A7000818085A26F5397E530D7E52C87E52C87E52C87E52C87E52C87E5229
S12352A0C87E52C87E52C87E52C87E52E87E52E47E52C87E52EC7E52CC7E52E07EE8E47E86
S12352C052D47E52D87E52DC86012024860220208603201C860420188605201486062010BB
S12352E08607200C8608200886092004860A2000B7020AB6020ABD525720F8BD520136A6E9
S12353000081042706BD52610820F43239F6102EB6102FC4082635F602252615812F261052
S1235320B60220B7022184EFB702208603B702253B7A02252608810D26181420043BF602C3
S1235340255A2604B702263BB702273B8601B702243B8602B702243B393939393C3736CED1
S123536003178630A100261B8D3F201DA10026198D378D3509A100261B8D2EA100261B8DF3
S123538028201DA600BDFFB808A600BDFFB8862EBDFFB808A600BDFFB808A600BDFFB808F4
S12353A0A600BDFFB83233383936088620BDFFB832393C3736EC00CE2710028FCB30F70316
S12353C0178FCE03E8028FCB30F703188FCE0064028FCB30F703198FCE000A02CB30F7030E
S10E53E01B8FCB30F7031A323338392F
S9030000FC
